:020000040000FA
:020000000029D5
:020008001A29B3
:1002000007309F0097010313831600308500FF30ED
:1002100086008312850186010930A000A1018316A2
:10022000053081008312F0308100A0308B00060879
:10023000A20019290B1121080339031D37290230A7
:100240002006031D252985142C29013020060319B9
:100250002C29201835298510A00B6129851022082A
:10026000A3001830A0002114612985142C29211C19
:10027000562921080C39031D472985142115A00B87
:10028000612985100430A0002110A1146129043ACD
:10029000031D5329A30C03184F29851050298514D9
:1002A0002111A1153F298510A1113F298514A00B0B
:1002B00061298510A1100930A0000608A20061295B
:0802C0000000F030810009008C
:00000001FF
